:020000040800F2
:2000000000200020210B0008150B0008170B0008000000000000000000000000000000001A
:20002000000000000000000000000000190B000800000000000000001B0B00081D0B000836
:20004000710B0008710B0008710B0008710B0008710B0008710B0008710B0008710B000880
:20006000710B0008710B0008710B0008710B0008710B0008710B0008710B0008710B000860
:20008000710B0008710B000800000000710B0008710B0008710B0008710B0008710B0008C4
:2000A000710B0008710B0008710B0008710B0008710B000800000000710B00080000000028
:2000C00010B5064C2378002B07D1054B002B02D0044800E000BF0123237010BD1800002077
:2000E00000000000380D0008044B10B5002B03D00349044800E000BF10BDC0460000000097
:200100001C000020380D0008002243088B4274D303098B425FD3030A8B4244D3030B8B42FE
:2001200028D3030C8B420DD3FF22090212BA030C8B4202D31212090265D0030B8B4219D334
:2001400000E0090AC30B8B4201D3CB03C01A5241830B8B4201D38B03C01A5241430B8B42BD
:2001600001D34B03C01A5241030B8B4201D30B03C01A5241C30A8B4201D3CB02C01A52411E
:20018000830A8B4201D38B02C01A5241430A8B4201D34B02C01A5241030A8B4201D30B02D4
:2001A000C01A5241CDD2C3098B4201D3CB01C01A524183098B4201D38B01C01A524143091B
:2001C0008B4201D34B01C01A524103098B4201D30B01C01A5241C3088B4201D3CB00C01A8E
:2001E000524183088B4201D38B00C01A524143088B4201D34B00C01A5241411A00D2014630
:20020000524110467047FFE701B5002000F006F802BDC0460029F7D076E770477047C0460E
:20022000F0B587B015006A46CC0F6418641063000733DB08DB00D31A00AF9D466E467860EC
:2002400022000021300000F06FFD00237868A34237DB2E4A01211300FC60D0680842FCD17D
:200260001169090605D52A4909685160294909685160AA0515D1196902320A431A6140227D
:200280005D6119690A431A610122D9681142FCD12022D968114200D0DA6002211A698A437F
:2002A0001A61002220203A617A6101327C69F9688C4211D38022BD4619690A431A6107B01A
:2002C000F0BD4278120294466146027802300A43590072520133BAE71969114319617C6902
:2002E00039696400A45B49190C80D9681142FCD1D968014200D0D8601969914319613969AC
:2003000002313961796901317961CFE7002002400000002004000020002310B5934200DB2E
:2003200010BDCC5CC4540133F8E7000010B5102488B02200002104A800F0F6FC80200A4AA7
:20034000C002516901435161536902A903400193019B00230548039301330294069300F0F8
:2003600008FC08B010BDC046001002400004004880230022DB055A625A6A8242FCD37047E1
:2003800010B572B6094B0A4A1B681360094A1278012A03D00022084B1A8010BD074A136057
:2003A000074A126882F308889847F6E70410000858010020007C00084200002068020020AC
:2003C00000100008F7B50191002100900B0008000125124A124F11705170019C84420BDC94
:2003E000002902D013701B0A537011780D4B197052780D4B1A70F7BD00990C5C082126007D
:200400005E405B082E4201D07B409BB20139C9B264080029F3D129000130DEE73400002011
:2004200001A0FFFF5E0100205D01002070B54318455C5C78FFF7C6FF054B00201B78AB4280
:2004400005D1044B1878001B43425841C0B270BD5E0100205D01002010B5FFF767FF0022CF
:20046000014B1A6010BDC046700200200449054A0B681A4080235B0013430B607047C0466C
:2004800000040048FFFCFFFFF8B500231D4D80202B701D4B10221F00C0051969114223D05C
:2004A0001A4B802019781023C0053A6914001C401A4221D11A20FFF75BFF01263420FFF752
:2004C00057FF3B692A781B093340A340013413432B70082CF2D11A20FFF74AFF0B4B2A7878
:2004E0001E700B4B1A7006E0446A0A498C42D4D96522094B1A80F8BD426AFA2AD5D900295B
:20050000D3D0F8E74700002000040048460000206E020020400D030042000020F8B510271A
:20052000060008250A4CA7623420FFF721FF01231E420BD0A761013DEDB27608002DF3D10C
:200540003420FFF715FF1023A361F8BDA762F2E70004004810B5FFF789FF3020FFF7DEFFBD
:20056000FFF77AFF10BD10B5FFF780FFC120FFF7D5FFFFF771FF10BD10B5FFF777FFC22014
:20058000FFF7CCFFFFF768FF10BD70B506000D000024AC4200DB70BD305DFFF7BFFF342089
:2005A000FFF7E6FE0134F4E710B5FFF75FFF09210248FFF7EAFFFFF74FFF10BD08000020AC
:2005C000F7B5904D904C2B7800AF002B21D08F4B200019888E4B1980FFF728FF002815D011
:2005E00080228C4E52000021300000F09DFB884B1A8800239A4205DCFFF7ACFF00232B70A0
:20060000BD46F7BDE15CF1540133F3E7FFF7B4FFF6E7814B21781960237C7D2B0AD1237A70
:200620000D2BEDD1637A422BEAD1FFF7BDFF00232375E5E7237D7D2B05D1237B0D2B02D1BF
:20064000637B422BF1D0230028331B787D2B07D1631CDB7F0D2B03D1A31CDB7F422BE4D0DE
:20066000002912D1A27863781343E278134302D165226A4B1A80FFF7F9FEC120FFF74EFFB9
:20068000664A13880133138048E0012917D1604B013120001980FFF7C9FE0028B6D0604B62
:2006A0001A68604B9A4202D8FFF75DFFA8E7574B58481988FFF7B4FDFFF74CFFA0E7FF29FC
:2006C00016D1534BFB3920001980FFF7AFFE00289CD00022514B1A80E378A2781B02134331
:2006E00080225BBA12059BB29B184D4A1360E3E7FE2919D1464BFA3920001980FFF796FE40
:20070000002883D0A378012B0BD0E3783F4A1380012380222B70444B52001A80FFF79CFE59
:200720006EE780235B00F1E7FD290ED1384BFB3920001980FFF77AFE002800D166E7FFF76F
:2007400095FEC120FFF7EAFEE8E702290DD1304B20001980FFF76AFE002800D156E7304A2D
:20076000304B12689A429FD9A6E704293AD101222E4B1A707FE72E4A136801331360647869
:20078000002C01D10134FF348022274BE51C1A80FFF76CFE23006A460A33DB08DB00D31A29
:2007A0009D462A00002168467B6000F0BDFA1C4B220019686846FFF7AFFD21006846FFF7BC
:2007C00001FE1C4B7A681B78290013551A4B6C441B78684663703023A370FFF7D6FEFFF75E
:2007E0003BFE0DE0032900D045E70221084B20006E461980FFF71AFE0028BCD1FFF7BCFE55
:20080000B546FDE6410000205F010020480000206C0200204A0000203800002042000020FF
:200820004C010020FF0F000862020020400000203C0000205E0100205D010020F8B58122A8
:2008400000241B4D1B4E1C4B210028008027520034601C7000F068FAFF05FFF715FE174B19
:200860001B78002B11D0164A3368128802329A420FD0144A0133127833602A708123013433
:2008800001355B009C42E8D103E07A6AFA2A03D93360FFF795FEF8BD0A4B1B782B700223F0
:2008A000FF339C42EAD1084A138814331380E5E75F0100203C000020460000204100002037
:2008C00048000020470000204200002010B50A4C302220000949FFF71FFDA3780B2B0AD0CB
:2008E000013BDBB2FD2B06D80B2330212000034AA370FFF795FC10BD5F010020007C0008D2
:20090000F8B58023FA201D4C1D4EE2689B0032401343FA27E3604000FFF72AFD10257F0077
:2009200023692B4203D1174A1388013313800A20013FFFF71DFD002FF2D1124D2B88002B7E
:200940001BD0FA20E3682F801E40E6604000FA26FFF70EFD7600103723693B4202D12B8847
:2009600001332B800A20013EFFF702FD002EF3D12B88002B01D0FFF703FDF8BD00040048A2
:20098000FFFCFFFF440000200122234910B50B68934313430B600B68204B19680A431A6076
:2009A000022219681142FCD0F8211A688A43110080220A431A605A6819491140A0229203C5
:2009C0000A430F215A60DA6A8A43DA628022196852040A431A608022920419681142FCD07B
:2009E000F0215A688A435A605A680E490A4003215A605A688A43110002220A430C215A6064
:200A00005A680A40082AFBD1074800F053F9064800F060F910BDC046002002400010024023
:200A2000FFFFC2FFFFF8FFFF006CDC0270B501258021304C88B0A36949052B43A361A36940
:200A400003AE2B400193019BE2690A43E261E369294A0B400093009B102311680B431360CA
:200A6000FFF792FF14220021300000F05DF9E36901222B43E361E36980242B400293029B74
:200A80002F2333800023E4055242310020007360B260F36000F0BEF880222368174993431F
:200AA0002360A3680B407021A36063688B436360A3689343A36023681D432560FFF736FCF1
:200AC000FFF71EFF0E490F4ACB681A4080235B001343CB600C4B1A780C4BDA70FFF7F6FED3
:200AE000FFF7ACFE0A4B1B88642BF9D9FFF748FCF6E7C0460010024000200240F8BFFFFF77
:200B000000040048FFFCFFFF1100002008000020420000207047FEE770477047704770475D
:200B20000D4885460D480E490E4A002302E0D458C4500433C4188C42F9D30B4A0B4C0023D0
:200B400001E013600432A242FBD3FFF7E8FF00F0C7F8FFF76BFFFEE7002000200000002028
:200B600018000020580D00081800002074020020FEE7F7B500254B680A680093013B0193C4
:200B80001300EB400AD1019B012B05D84368C96893434A431A4342600020FEBD0124130046
:200BA000AC402340224228D01A0003275A4357433E000468FF43B443009E5643344304601A
:200BC000019C012C05D88C68866854433E40344384600C69C668544337402743009CC7603E
:200BE000022C0AD14C69FF2B09D80F26524356436243036AB343134303620135BBE70F22FD
:200C00001B0A5B435B435A436343466A96431E434662F2E7204A10B50368904206D08024DF
:200C2000E405A04202D01D4CA0420CD17024A3434C682343904212D08024E405A0420ED05A
:200C4000164CA0420BD0164CA04208D0154CA04205D0154CA04202D0144CA04203D1144CB6
:200C60002340CC68234303608B68C3620B888362904208D00B4B984205D00B4B984202D0D3
:200C80000A4B984201D10B7C03630123426913434361002010BDC046002C014000040040F9
:200CA00000200040004001400044014000480140FFFCFFFFFA2110B58900FFF725FA0022AC
:200CC000034B013858609A6005321A6010BDC04610E000E0014B18607047C04614000020D2
:200CE00070B500260C4D0D4C641BA410A64209D1002600F021F80A4D0A4C641BA410A6420B
:200D000005D170BDB300EB5898470136EEE7B300EB5898470136F2E7500D0008500D000840
:200D2000500D0008540D000803008218934200D1704719700133F9E7F8B5C046F8BC08BC23
:200D40009E467047F8B5C046F8BC08BC9E467047E9000008C100000823016745AB89EFCDB8
:200D6000343731001F0606013014000000127A0000000000000000000000000000000000DB
:200D8000000000000000000000000000000000000000000000000000000000000000000053
:200DA000000000000000000000000000000000000000000000000000000000000000000033
:200DC000000000000000000000000000000000000000000000000000000000000000000013
:200DE0000000000000000000000000000000000000000000000000000000000000000000F3
:200E00000000000000000000000000000000000000000000000000000000000000000000D2
:200E20000000000000000000000000000000000000000000000000000000000000000000B2
:200E4000000000000000000000000000000000000000000000000000000000000000000092
:200E6000000000000000000000000000000000000000000000000000000000000000000072
:200E8000000000000000000000000000000000000000000000000000000000000000000052
:200EA000000000000000000000000000000000000000000000000000000000000000000032
:200EC000000000000000000000000000000000000000000000000000000000000000000012
:200EE0000000000000000000000000000000000000000000000000000000000000000000F2
:200F00000000000000000000000000000000000000000000000000000000000000000000D1
:200F20000000000000000000000000000000000000000000000000000000000000000000B1
:200F4000000000000000000000000000000000000000000000000000000000000000000091
:200F6000000000000000000000000000000000000000000000000000000000000000000071
:200F8000000000000000000000000000000000000000000000000000000000000000000051
:200FA000000000000000000000000000000000000000000000000000000000000000000031
:200FC000000000000000000000000000000000000000000000000000000000000000000011
:200FE000000000000000000000000000000000000000000000000000000000000BFFFFFFE9
:20100000004000201D590008BD690008C16900080000000000000000000000000000000092
:20102000000000000000000000000000C56900080000000000000000C9690008CD69000802
:201040006D5900086D5900086D5900086D5900086D5900086D5900086D5900086D59000820
:201060006D590008CD6A0008D16900083D6A0008416A0008F56A00086D5900086D590008BC
:20108000A96A00084D6A000800000000696A0008856A00087D6A00086D5900086D59000819
:2010A0006D5900086D5900086D590008816A00086D590008000000006D5900080000000037
:2010C000015C417264754265652020202020000010B5064C2378002B07D1054B002B02D079
:2010E000044800E000BF0123237010BDBC01002000000000D0710008044B10B5002B03D049
:201100000349044800E000BF10BDC04600000000C0010020D0710008002243088B4274D31A
:2011200003098B425FD3030A8B4244D3030B8B4228D3030C8B420DD3FF22090212BA030C1A
:201140008B4202D31212090265D0030B8B4219D300E0090AC30B8B4201D3CB03C01A524125
:20116000830B8B4201D38B03C01A5241430B8B4201D34B03C01A5241030B8B4201D30B03DE
:20118000C01A5241C30A8B4201D3CB02C01A5241830A8B4201D38B02C01A5241430A8B42F8
:2011A00001D34B02C01A5241030A8B4201D30B02C01A5241CDD2C3098B4201D3CB01C01AC7
:2011C000524183098B4201D38B01C01A524143098B4201D34B01C01A524103098B4201D303
:2011E0000B01C01A5241C3088B4201D3CB00C01A524183088B4201D38B00C01A5241430863
:201200008B4201D34B00C01A5241411A00D20146524110467047FFE701B5002000F0F0F8CD
:2012200002BDC0460029F7D076E7704703460B437FD4002243088B4274D303098B425FD36F
:20124000030A8B4244D3030B8B4228D3030C8B420DD3FF22090212BA030C8B4202D312123E
:20126000090265D0030B8B4219D300E0090AC30B8B4201D3CB03C01A5241830B8B4201D39B
:201280008B03C01A5241430B8B4201D34B03C01A5241030B8B4201D30B03C01A5241C30AB2
:2012A0008B4201D3CB02C01A5241830A8B4201D38B02C01A5241430A8B4201D34B02C01A16
:2012C0005241030A8B4201D30B02C01A5241CDD2C3098B4201D3CB01C01A524183098B42B5
:2012E00001D38B01C01A524143098B4201D34B01C01A524103098B4201D30B01C01A524155
:20130000C3088B4201D3CB00C01A524183088B4201D38B00C01A524143088B4201D34B00CE
:20132000C01A5241411A00D201465241104670475DE0CA0F00D04942031000D340425340C0
:2013400000229C4603098B422DD3030A8B4212D3FC22890112BA030A8B420CD38901921197
:201360008B4208D3890192118B4204D389013AD0921100E08909C3098B4201D3CB01C01A38
:20138000524183098B4201D38B01C01A524143098B4201D34B01C01A524103098B4201D341
:2013A0000B01C01A5241C3088B4201D3CB00C01A524183088B4201D38B00C01A5241D9D241
:2013C00043088B4201D34B00C01A5241411A00D20146634652415B10104601D34042002B77
:2013E00000D54942704763465B1000D3404201B5002000F005F802BD0029F8D016E7704746
:201400007047C046844608006146FFE71FB500F06DFB002801D40021C8421FBD10B500F0CB
:20142000F9FA4042013010BD10B500F05FFB002801DB002010BD012010BDC04610B500F090
:2014400055FB002801DD002010BD012010BDC04610B500F005FB002801DC002010BD01208D
:2014600010BDC04610B500F0FBFA002801DA002010BD012010BDC0469E2110B5C905041C99
:20148000FFF7F0FF002803D1201C00F047FE10BD9E21201CC90500F093FC00F03FFE802315
:2014A0001B069C466044F2E7F0B5C64643025B0A4E0245004F00DA00C40F9C46700A90468E
:2014C00000B52D0E3F0EC90FB6098C424BD0EA1B002A36DD002F61D0FF2D00D1ADE0802380
:2014E000DB041E431B2A00DCD3E001204346181A430100D48CE080018709380000F0BEFE83
:2015000005388740854200DCB6E02D1AB3483840430704D00F230340042B00D004304301CA
:2015200000D478E06A1CFE2D65D08001430A9C46D2B26346D0051843E407204380BCB84604
:20154000F0BD002A35D07A1B002D00D0AFE04346002B00D1A7E0531E012A00D12FE1FF2ADC
:2015600069D01A00AAE0E91B002970DD002F37D0FF2D62D08023DB041E431B2900DCB0E0ED
:2015800001204044430143D50135FF2D33D00123934A0340400810401843B9E7002E00D10F
:2015A00083E0511E012A00D1D8E0FF2A45D00A0098E7FE276A1C174200D086E0002D00D0A7
:2015C000B7E04346002B00D1F3E00022002EB0D0981B430100D4FAE043460C00F01A97E78A
:2015E000002E00D1C8E04A1E012900D1AEE0FF2923D01100C1E70023FF229C4699E7FE21BA
:201600006A1C114277D0FF2AF5D0150046447008430700D07EE7C308FF2D0ED05B025B0A8F
:201620009C46EAB285E7002E07D08022D203134203D0104201D10C000300002BDBD0802073
:20164000C00318434002430A9C46FF2271E70029D5D07A1B002D60D14346002B24D0531EA8
:20166000012A73D0FF2AE7D01A001B2A00DC85E001203D00801985E720233A00451B380004
:201680000135EA405D1BA840431E9841002510433EE7202330009B1A31009840D140431E10
:2016A0009841084322E70C0003001500B4E7FF2FC1D080234046DB04184380461B2A51DDE3
:2016C00001200C003D00301A12E743469F1B7B012BD4002F00D010E70023002400229C465E
:2016E00027E7202332003000CA40591A8840431E9841104345E7002D4AD14346002B63D00A
:201700000022002E00D114E730004044430100D47EE7324B013518407AE7FF2F8CD08023E3
:201720004146DB04194388469FE743460C00F71AE3E64246002A00D075E7002E00D07AE7E7
:201740008023DB0300249C46FF22F2E6300040440125430100D45BE7022518E74346012500
:20176000981BC5E6202344464046D4409A1A9040431E98412043A4E70D004DE720234146ED
:201780004046D1409A1A9040431E9841084370E74246002A00D14FE7002E00D14DE78022C4
:2017A000D203134200D148E7104200D045E7030043E7002E90D00C0084460022B9E64346D6
:2017C0000C00F01A013593E684460022B1E6002800D01DE7002300249C46AAE6FFFFFFFB14
:2017E000FFFFFF7DF0B54F464646D6464502C0B547000C1C6D0A3F0EC60F002F00D170E079
:20180000FF2F00D175E0EB008025ED041D43002399469A467F3F6002430A984663001B0EDA
:20182000E40F002B4ED0FF2B46D04246D0008022D2040243904600227F3B3100FF1A4B468A
:201840006140C9B213430F2B00D9B5E06E489B00C3589F46002398462600454692465346FA
:20186000022B00D189E0032B00D19EE0012B18D03B007F33002B69DD6A0704D00F222A4032
:20188000042A00D004352A0103D5604B1D403B008033FE2B00DD70E0AD016D0AD8B202E031
:2018A0000E0000200025C0052843F6073043E0BCBA46B146A846F0BD4346002B3FD102221F
:2018C000FF3F03E04346002B2DD1012231004B466140C9B213430F2B34D84D489B00C3584D
:2018E0009F46002D13D104239946033B00279A4691E7002D05D108239946063BFF279A46DB
:2019000089E70C239946093BFF279A4683E7280000F0B4FC7627431F9D4000237F4299462E
:201920009A463F1A77E7404600F0A8FC4246431F9A4076235B4290461B1A00227DE7FF2349
:2019400003227AE70E00FF200025ACE70120C01A1B28A6DC9E372A00BD40C2406B1E9D41F7
:2019600015436B0704D00F232B40042B00D004356B0144D50120002595E7FF20002592E7F0
:2019800080250026FF20ED038DE7002398468020C003054209D04346034206D145460543FD
:2019A0006D022600FF206D0A7DE78020C00305436D02FF206D0A76E742466B015001834281
:2019C00019D21B220025013F01261C006D005B00002C01DB984201D81B1A3543013A002AA2
:2019E000F3D15A1E93411D433B007F330E00002B00DD41E7AAE71A2201251B1AE4E7AD01AB
:201A000000206D0A4FE7C046E8710008FFFFFFF72872000870B5420045024E024C00C30FE0
:201A20006D0A0120120E760A240EC90FFF2A06D0FF2C03D0A24201D1B54206D070BD002D8A
:201A4000FCD1FF2CFAD1002EF8D18B4206D00120002AF3D12800431E9841EFE70020EDE7EE
:201A600070B5420045024E024C00C30F6D0A120E760A240EC80FFF2A1BD0FF2C0ED0002AE3
:201A80001BD1002C01D1002E1CD0002D0CD083421CD00221581E0840013870BD002E22D120
:201AA000002AF4D1002DF2D10028F6D101204042F3E7002D17D1FF2CF0D0002CE7D1002EC9
:201AC000E5D1E6E70020002DE7D0E2E7A24205DCEADBB54202D8E7D30020DEE7434258419E
:201AE00040000138D9E702204042D6E770B5420045024E024C00C30F6D0A120E760A240EE7
:201B0000C80FFF2A0BD0FF2C0DD0002A1FD1002C16D1002E14D10020002D10D009E0002D5F
:201B20000CD1FF2C13D1002E08D1002A08D0834212D00221581E0840013800E0022070BDC0
:201B4000002DF4D10028FAD101204042F7E7002CEDD1002EEBD1ECE7A24205DCF2DBB542EF
:201B600002D8EFD30020EAE74342584140000138E5E7C046F0B54F464646D6464402450002
:201B8000C0B5640A0F1C2D0EC60F002D00D18DE0FF2D00D192E00023802099469A46E400E7
:201BA000C00404437F3D7802430A98467B001B0EFF0F002B00D170E0FF2B00D186E04246D2
:201BC000D00080227F3BED180023D204024390469C4631004B467940681C0F2B1CD8764AF1
:201BE0009B00D3589F4639004446E2465346022B0FD0032B00D1D7E0012B37D1002000247C
:201C0000C0052043C9070843E0BCBA46B146A846F0BDFF200024F3E7260C2404220C444624
:201C20002404240C434627001B0C574374435A435E4312193B0C9B189C4203D98022520211
:201C4000944666443F041A043F0CD2199401671EBC411B0C920E9B1914439B011C431B0169
:201C600000D49BE0012362081C40144302007F32002A64DD630704D00F232340042B00D0E4
:201C80000434230103D502004C4B80321C40FE2ABFDCA401640AD0B2B2E74346002B3DD1B6
:201CA0004A4601331A4391469C4692E7002C29D104239946033B00259A4674E7002C1BD1EF
:201CC00008239946063BFF259A466CE74346FF35002B0BD102234A461A4391469C4678E774
:201CE00053463100022B00D083E792E703234A461A4391469C466CE70C239946093BFF25A5
:201D00009A4650E7200000F0B9FA7625431F9C4000236D4299469A462D1A44E7404600F097
:201D2000ADFA4246431F9A4000232D1A90469C46763D4EE780240021FF20E40360E70123F8
:201D40009B1A1B2B00DD59E722009E30DA4084401300621E94411C43630704D00F23234003
:201D6000042B00D0043463011AD50120002447E78020C003044209D04346034206D14446B5
:201D8000044364023900FF20640A39E78020C003044364023100FF20640A31E7280065E756
:201DA000A4010020640A2BE78020C00304436402FF20640A24E7C04668720008FFFFFFF75A
:201DC000F8B5CE46474643025B0A4E02DA009446720A914645004A0080B52D0E1F00C40FC3
:201DE000120EC90FB609FF2A5BD0012041408C4239D0A81A00285ADD002A6AD0FF2D00D1DD
:201E0000D9E08022D20416431B2800DCE9E001206346181A430100D4B4E08001870938005F
:201E200000F02CFA05388740854200DCCCE02D1AB5483840430704D00F230340042B00D0EB
:201E40000430430100D4A0E06A1CFE2D00D18DE08001470AD2B2D0053843E4072043C0BC57
:201E6000B946B046F8BDA81A8046002845DD002A70D0FF2D00D19EE08023DB041E43434695
:201E80001B2B00DCD2E00120604443017AD50135FF2D6BD001239D4A034040081040184338
:201EA000C8E7002E20D08C4223D02800FF38002839D0571B002D00D09DE06346002B00D173
:201EC000DBE07B1E012F00D10DE1FF2F71D01F0098E0002E00D1A7E0421E012800D1E6E013
:201EE000FF2868D010008FE701204140A14200D07FE7FF2040428046A8444046002838D039
:201F0000511B002D00D1AEE0FF2A00D1DFE080236046DB04184384461B2900DCD9E00120C9
:201F200015008019B1E7FE206A1C104271D1002D00D0A6E06346002B00D1D9E00022002EF2
:201F400000D188E7981B430100D4E1E063460C00F01A6FE7002E00D1B7E00200013A0128A4
:201F600000D19CE0FF2826D0904688E7FF22002771E7FE206A1C104264D0FF2AF6D01500E4
:201F800066447008430700D056E7C308FF2D12D05B025F0AEAB25EE76246002A00D196E02F
:201FA000002E08D08022D203134204D04846104201D10C004B46002BD8D08027FF031F434E
:201FC0007F02FF227F0A46E720233A00451B38000135EA405D1BA840431E98410025104322
:201FE00028E720231B1A32009E40C2403000431E984110430CE7FF2ADBD080236046DB049C
:20200000184384461B2F56DD01200C001500301A00E763469F1B7B013DD4002F00D0FEE6D8
:2020200000240022002716E70500AFE7320043464146DA4020235B1A9E403000431E98413F
:20204000104321E7002DA7D16346002B59D00022002E00D1FFE630006044430192D52A4B89
:20206000013518408EE76346002B47D04B1E012915D0FF292BD019004EE70C004B463D00AF
:2020800084E76246002A8BD1002E92D180270024FF22FF03DFE663460C00F71ABFE63000C8
:2020A00060440125430100D46CE70225F2E663460125981BAEE6202364466046FC40DF1B0D
:2020C000B840431E984120439FE705005EE74B4671E7202365466046CD40591A8840431E75
:2020E000984128431CE763460C000125F01A91E6002E95D00C004F460022ACE64B460D00B7
:2021000044E74F460022A6E6FFFFFFFBFFFFFF7D002800D036E7002400279CE64102420078
:20212000C30F490A0020120E7E2A03DD9D2A02DD094A98187047802000040143952A07DCC8
:202140009620821AD1404842002BF3D10800F1E7963A9140F7E7C046FFFFFF7FF8B50028ED
:2021600013D0C317C6185E40C40F300000F086F89E2305001B1A962B0FDC082801DD083DBB
:20218000AE407602760AD8B202E0002400200026C0053043E4072043F8BD992B0CDD052274
:2021A0003100121AD1400A00010030001B318840411E884102431600052D12DC31000D4F32
:2021C0003940720709D00F203040042805D004314A0102D59F2339405B1B89014E0AD8B220
:2021E000D6E76A1F96403100024F39407207F4D0E9E7C046FFFFFFFB70B5051E0ED000F0A7
:202200003DF89E2304001B1A962B0CDC082801DD083CA5406D026D0AD8B201E00020002519
:20222000C005284370BD992B09DD020029001B3291404A1E91410522121AD5400D43052C2B
:2022400012DC29000C4E31406A0709D00F202840042805D004314A0102D59F2331401B1BFA
:2022600089014D0AD8B2DBE7621F95402900024E31406A07F4D0E9E7FFFFFFFB1C21012393
:202280001B04984201D3000C10391B0A984201D3000A08391B09984201D30009043902A242
:2022A000105C40187047C0460403020201010101000000000000000070B500260C4D0D4C91
:2022C000641BA410A64209D1002604F081FF0A4D0A4C641BA410A64205D170BDB300EB58AE
:2022E00098470136EEE7B300EB5898470136F2E7447300084473000844730008487300080E
:2023000003008218934200D1704719700133F9E73B49F0B50A88002A3BD00020130008807B
:20232000100A110941404A400F2108001B019043344A03431360344A1813145C0800184087
:20234000105CE403044318121B1108400B40105CD35C40220125800204435B011C432B4BDD
:202360002B4F1C602B4B1E78731C9B00B600FA50B81941682D3A2B0093402340D34089094A
:202380005940890181600430013AF4D20023BB51F0BD214B1B78002B1AD0204B1B68D9133A
:2023A000012918D0991301291ED0591301291DD0191301291CD0D91201291BD099120129AD
:2023C0001AD05912012919D015490A609AB2A7E7144B124A13600F22083A134110490A603B
:2023E00051020B439AB29BE70E22F5E70D22F3E70C22F1E70B22EFE70A22EDE70922EBE753
:20240000C60200202402002000730008C00200202C020020402B0020F40300201803002006
:20242000C8020020FFFF0000F0B5DE4657464E464546BC4BBC48DC6F1968E0B5621A92B203
:202440000280BA4889B084466244C62A00D996E05A689D68511A48090200D968B4481E69C7
:20246000026001924A1B5D695109AA1BDD699E691F6A416002915109AA1B5E6A5509F21BC1
:202480005609DF6A9A6A8160BF1A03911A6B790907975F6BC560BF1A7A098261049506923E
:2024A0009D6BDA6B0661521B52094161C261944605965A6C1D6C9E6E521B52099D6C904664
:2024C0000262DA6C1F6F521B520991461D6D42625A6D521B52099D6D93468262DA6D521BED
:2024E00052091D6E9246C2625A6E521BDD6E5209AE1B5D6F9B6FED1BE31A5B0976096D0922
:20250000059C026346638563C363019847466040029C784061404C4661406446C00089001B
:2025200001430498D2006040544660400143069C0398B60060405C4632431A437D4B60405C
:2025400040006D001B78154301437B4AC9B2EDB2002B1BD1107800281BD178480069C0051F
:2025600007D5774C20780130C0B22070642800D974E08D4212D0734A13880133138009B0AF
:20258000F0BCBB46B246A946A046F0BD1278002AEFD00F22551BEDB28D42ECD100216A4A00
:2025A00011806A490A8801320A805246012A02D15146674A1170019A0299920249020A43C7
:2025C00059460A430399079809020A430499C9010A43059989010A431F2188430699024364
:2025E0000F0161463A43CF0041463A438F0049463A4349000A432F2A1EDC511E2E2923D88F
:2026000000205449544CD2B208802270534909780029B4D1002BB2D0514B197891422AD04D
:202620001A70042A32D84F4900230B70152A1CD84D4B92009B589F46464B1A800023464A8F
:202640001370484A13709AE7002A64D1002341490A80414A1370434A137090E70120107095
:2026600097E7424B1A78424B1A702278414B1A700023237083E73B49042AD5D90B780133BF
:20268000DBB20B70052B00D879E7CDE70122354B1A7074E7354B1A7801239B1A344A1370A2
:2026A000E3E70022344B1A70344B354A1A80FFF72FFEDAE70122304B1A70E0222F4B1201F2
:2026C0001A80FFF725FED0E700F0BEFACDE701222C4B1A70C9E700222A4B1A70C5E7012270
:2026E000224B1A700022224B1A70274B02321A70BBE700221D4B1A7001231D4A1370224A6A
:202700001370B2E703F0C4F8AFE702F0BFFFACE703F002F8A9E7104C2278002A00D075E74C
:202720002DE7C046442B00202002002081FBFFFFDC010020E60200201403002000040048AC
:20274000C40200201C020020F803002028020020F5030020E803002015030020F40300207E
:20276000C5020020D8010020A87200081003002010010020E20300201E020020C6020020C6
:20278000FF0E0000F8020020F203002010B51C00884200DA08001300824200DD030002981F
:2027A0005B1A001B5843511AFEF740FD001910BD0300401A00D5C81A7047C0460023034A2A
:2027C0005362536A8342FCD37047C0460048014000230121084A5362084B936253690B430F
:2027E0005361536A8342FCD330230121936253690B4353617047C0460048014080BB00002B
:20280000BFF34F8F034B044ADA60BFF34F8FC046FDE7C04600ED00E00400FA05F8B5194DEF
:2028200003F078FAEB68184AFA201A408023FA2480279B021343EB608000FFF7BFFF134ECF
:20284000A4007F002B693B4211D133880A200133013C3380FFF7B2FF002CF3D1094A0A491C
:20286000D3680B40D3603388052B07D9F8BD0A20013CFFF7A3FF002CE4D1EFE702F0EAF994
:20288000FFF7BEFF00040048FFFFFCFFE6030020F0B5C64600B5B64CB0222000B54982B0AD
:2028A00003F000FA637CB44E013B5A425341B34A1370A37C013B5A4253413370E37C012BA5
:2028C00001D1AF4A1370637D013B5A425341AD4A1370A37D013B5A425341AB4A1370E37D80
:2028E000032B00D90223A94A1370207E0300083B282B1FD8103B182B00D811E103000C3B66
:20290000A34D0B2B00D81AE10300083B032B00D823E128889F4BD8629F4B18809F4B188096
:20292000607E0300323B642B0ED99D4B188840080A3017E09B4B9C4A1380964AD362607E80
:202940000300323B642BF0D8FA21914B40081B8804305843C900FEF769FC80B20200934BCA
:202960000A321A802822924B924D18809846A37E914F534314332B80E37E05203B70237FA9
:20298000013B5A4253418D4A1370637F013B5A4253418B4A137002F077FD6378002B14D17A
:2029A0002C889621874B20000093874A874B4900FFF7ECFE864B1880864B1B78002B00D192
:2029C000337002B080BCB846F0BDA07F0B2800D9A2E002F059FDE37F013B5A4253417E4A30
:2029E00013702023E35C7D4A7833FF335B0013807B4A21239446E35C7A4A63445B001380C5
:202A0000794A22239446E35C784A634413802323E25C774B1A702423E35C013B5A425341D7
:202A2000744A13702523E35C734AFA3313802623E35C013B5A425341704A13700022704B43
:202A40001A702823E35C5A1F142A01D86D4A13702923E35C5A1E092A01D86B4A13702A2304
:202A6000E25C531E082B1BD84146684B1A7053019B1A9B009B1A5B00654A5D3BDBB21370B2
:202A8000627E52089A180A8062490A889A180A8061490A889A180A803E4A516C0B43536485
:202AA0002B23E35C1A00463A462A01D85B4A13702C23E35C5A1E622A05D8594A5B0013807E
:202AC0000122584B1A702D23E35C5A1E092A01D8554A137096232C885B009C4202D20022D5
:202AE000524B1A7039782020FEF7A0FB642105002000FEF711FB290080B2FEF797FB4C4B0A
:202B0000112118802000FEF707FB290080B2FEF78DFB484B188044E7052002F0B5FC5AE79D
:202B2000454B3022009318211E4BFFF72FFE184D2880207E03000C3B0B2B00D9E4E6194B29
:202B4000182200930C213D4BFFF720FE2880207E0300083B032B00D9DBE6394B1022009342
:202B60000721384BFFF712FE80B22880D2E6C04620030020007C0008F802002010030020F8
:202B80000D040020D000002092010020D1000020CE000020002C0140940100200801002037
:202BA00020010020CF0700009801002088010020220100202401002026010020F9020020B2
:202BC000FA030020E2040000B80B0000C409000028010020DA000020DC02002030010020D0
:202BE0006B0300002E0100205E050000320100202C010020CC02002014010020D4020020FC
:202C0000DD02002034010020050100200601002004010020960100208C010020CC0000209E
:202C2000C00000200C04002035010020180100201601002012010020E70300009E0F0000F4
:202C4000B50B00006D17000010B5154B15481B78B0214370144B1B78013B5A425341437482
:202C6000124B1B78013B5A4253418374104B1B78013B5A425341C3740E4B1B78013B5A42AC
:202C8000534143750C4B1B78013B5A42534183750A4B0B4A1B78C37502F07AFF10BDC046E7
:202CA0000A0100202003002010030020F80200200D040020D000002092010020D100002094
:202CC000007C0008F0B5CE46474680B5C7480378012B5FD0042B5DD0C54D022B00D1AAE01A
:202CE000052B00D1A7E0032B00D1F4E0062B00D1F1E02B880420BF4A9168084204D19168B5
:202D0000BD4C2140014391600821BA4802681142FCD0BA4ABA485168BA4A521A92B2111CC0
:202D2000824200D9011C88B2CA0701D5013880B2984201D200232B80984200D844E1B24A3F
:202D4000002794461688B14A1278002A00D00FE19021C90589461021AD4A88460CE0012B09
:202D600005D9591E4900515AA14200D931E102339BB2984200D823E15900545A591C49003F
:202D8000515AA142EBD94746494601368F62B6B20127E4E700219F4A5156022900D11FE195
:202DA00002231370934A944993680B4010210B43936093681942FCD104228E498B681A428A
:202DC000FCD101228D490B6893430B6014000B681C401A42FAD1904B8A4D5A604B681B0C29
:202DE0001B042B434B600B681A430A600C22814B9A628A4B8A4A19680623914209D8894B90
:202E00001A68C8235B009A4264417D22634293438433854A78491380844A754D1380754A93
:202E200093680B4004210B43936000232B800378022B00D054E70023764AD356002B00D15D
:202E400057E7002313706B4A6B4993680B4010210B43936093681942FCD1042265498B6883
:202E60001A42FCD1012265490B6893430B6014000B681C401A42FAD1674B624E5A604B68CB
:202E80001B0C1B0433434B600B681A430A600922584B9A62614B624A19680623914209D811
:202EA000604B1A68C8235B009A4264417D226342934384335C4A504913805C4A13804D4AAB
:202EC00093680B4004210B43936000232B800378032B00D00AE700224E4B9A56012A00D167
:202EE00007E701221A70434A434993680B4010210B43936093681942FCD104223D498B68A4
:202F00001A42FCD101223D490B6893430B6010000B6818401A42FAD13F4B3A4C5A604B68AC
:202F20001B0C1B0423434B600B681A430A600A22304B9A62394B3A4A19680623914209D8F7
:202F4000384B1A68C8235B009A4240417D22434293438433344A28491380344A1380254A16
:202F600093680B4004210B43936000232B80C1E69021C905894610218846254A5900545A6D
:202F8000591C4900515A8C4207D9002905D0474649468F6101270136B6B2012B0CD9591EC1
:202FA0004900515A8C4207D9002905D049464446012701368C61B6B202339BB29842DDD893
:202FC000002F01D063461E802880C0BCB946B046F0BD49464446013601278C62B6B2C6E66A
:202FE000034D022B00D07BE62BE7C0468E010020E003002000240140E8FFFF7F0800024045
:203000008613000088130000F60200202B0100202C0400202701002000000240EC02002030
:20302000C4090000140400201C0100201E010020F8B5574D57482978574A00884E1E730076
:20304000985250881388554C1B1890881B18D0881B18108952891B189B185B102360504B86
:20306000187801282FD0F0B2002825D00123287019404C4B19704C4B1B78002B31D0FA2331
:203080004A4ADB0012689A4208D9494B494A1B781278134302D00122474B1A700022474B2B
:2030A0001A80474B1A70474B1B78002B03D0464B1B78002B1ED1F8BD06232B70434B0121D0
:2030C00018700620D5E70131C9B206290CD80200080029700A40334B1A70334B1B78002B95
:2030E000CDD101F0FFFDCAE70022384B28701A700132F0E7364B2068364C1B88A169A26881
:20310000C01A0B185343226920609446226A63442361934201DD1300226152429A4201DDE9
:2031200013002261421AE168A0614A436168626148438018C018636AE061984201DD180061
:20314000E3615B42834201DD1800E361FFF706F82149FEF747FB214E214F3168FEF7A4F9F0
:20316000391C051CFEF774F9002806D10027281C391CFEF759F9002807D03760194B1B68F4
:20318000632B98D80023236195E73560F6E7C0468E010020D8000020FC0200201803002096
:2031A000100100202B010020F3030020EC020020FA030020D4020020EA030020F602002036
:2031C000120400200E040020F40300200E030020020400203801002000401C46D403002027
:2031E00000E0FF44140400200121124A10B5D368114C8B43D360228853009B180F4A1288F5
:203200009B189B102380FFF713FF0D4A23881278D9084A430B4992B25B089B1A0A800A4A1D
:203220000A4913800A4A13688B4201D80133136010BDC04600200040D80000200A04002033
:20324000D1000020E4020020100400200F27000014040020F0B5DE4657464E464546784C8C
:20326000E0B52388774A01339BB287B0238093421AD9754B754D00269E5F3000FEF76EFFF3
:203280007349FEF7AFFA2968FEF70EF92860714D2B78022B00D10DE3032B00D15DE2012B06
:2032A00000D150E2002323806B4E6C4D33782A78134304D16A4A1178002900D007E3694B87
:2032C0000293694B1B78002B00D0A6E0674F684B9B461B78002B59D0664B674C9846674B6C
:2032E00003211868FDF7A2FF654D20602B78002B05D0644B99461B680A2B00D93CE24246FB
:20330000C82312885B009A422FD9C2225E4992008B585E480340FF208B5004328B58834327
:20332000BF3803438B503B78002B01D000233B70574A138801339BB21380029A1178554AE4
:2033400001314A43934209DD3478002C01D000F0FFFB514A934201D900F016FC07B0F0BCB1
:20336000BB46B246A946A046F0BDC221464889004358464A1A408023DB031343C322435004
:20338000FF21920083588B438350CCE7434B1A789A46434B188893009B181B012E33834296
:2033A00000DA95E03F4B404C0393324B98463F4B04933F4B99463F4D2B78002B09D0012BCE
:2033C00001D100F014FC022B01D100F015FC00232B70394B1B78002B00D0B9E24A4613808D
:2033E000039B1B78002B00D0E7E20121334A1170244A1360324B1B78002B00D0DBE2237874
:20340000002B01D100F067FC2E4B1B78002B01D000F048FC33789A46D9E22B482B4A038867
:20342000117801338A009BB25218104F03805200934200DC4BE701233B700023038046E7D5
:203440000804002010270000DE020020080300200000B4431E020020E6020020FB02002082
:20346000D2030020F6030020DC020020F503002000040020D8000020EC02002018030020C3
:203480000E0300201404002000E100E0FFFF00FFF8030020C4090000A86100000D040020E3
:2034A000D0030020F4030020F3030020E403002016030020F2030020DA000020EA03002090
:2034C000F9020020D402002004040020930100203378002B00D173E1CF4B03931B78002B96
:2034E00000D16CE3CD4B9846CD4B0493CD4B05931B88002A00D1FCE28921CB4A12880092F0
:20350000CA4AFFF743F9CA4B85B20A2120881D809946FDF787FE89B2002900D092E0C54B9B
:203520001B78002B00D1F3E2039B1B78002B00D188E06420C04B00229B5EC04A12885043B1
:20354000181ABF4B9C69996822184A43196918608C46196A62441A618A4201DD0A001961C4
:203560004942914201DD0A001961D968041B4C43596898614843001980185A6A5C61D861EC
:20358000904201DD1000DA615242824201DD1000DA61FEF7E3FDAB49FEF724F9FEF7BEFD24
:2035A000A94C059A238812881B1A1BB22380934201DA13B223809D4200DA2580A34B1B7896
:2035C000002B3FD043461888A14B1B88C01AA14B9C69996822184A43196918608C46196A17
:2035E00062441A618A4201DD0A0019614942914201DD0A001961D968041B4C435968986113
:203600004843001980185A6A5C61D861904201DD1000DA615242824201DD1000DA61FEF743
:203620009DFD8849FEF7DEF88B4B8C4C1968FDF73BFF211C0590FDF70BFF002800D161E3EA
:20364000854B1C60864B1B78002B00D040E2854C2370854B1A88534619788B005B181B0183
:203660002E339A4200DCA6E633789A46774B1A78142313417D4A126893420DD97C4B1B88D5
:20368000AB4202D94A461D0013807A4B1B88AB4202D24A461D001380774B1B88AB4202D293
:2036A0004A461D001380634B1B78002B07D0664B00229B5E9D4202DD9DB24B461D80664BCF
:2036C00000211C68201CFDF7C3FE002806D0201CFDF7D2FE4B462D18ADB21D80674B684C1E
:2036E0001B78002B1ED0FA2322685B009A4200D9EAE11E211E221E20624B1870049B18886B
:203700002B1A934200DCD6E14B464246401885B21D80FA2312885B009A4200D903E20022E9
:20372000594B1A705346002B00D038E1039B18784300C3189B00C018544B80B21880544BE7
:203740001B889B4659E0534B1A7880239B001343514A138002232B70A4E5504B19211888FC
:20376000FDF7DAFCFF2303408020C00018434A4B188001232B7095E5494B010018689A4604
:20378000FFF716F823685A08904214D9FA22D200934210D200214A4642481160027801327B
:2037A00002701D4A1170404A01311170304A1C49128852080A8000222A70524613609EE5CB
:2037C000284B1B789A46002B00D126E1134B9846134B0493164B9946134B19884B461D885A
:2037E0002B4B4C1C1B88180068439B46FDF71EFD264B201A80B2224C1880049B59461D80D7
:203800005B462A4AD3622A4BD96250639063D06358639863D86362E5F4030020D80000208E
:20382000E403002022010020CE000020FF070000160300200C040020DE020020C000002001
:20384000DC00002000401C469A010020FA0300208A01002060010020FC030020000016434E
:20386000D4020020F3030020D003002014040020200100208C010020080100201A010020BF
:20388000EC020020190100200E010020E0020020980100200D030020C6020020F2020020CA
:2038A000DC0300200F030020EA030020002C0140000400403221F0B2FDF72EFCC3B2C020B1
:2038C000C0001843CE4B188003232B70EAE4CD490988002900D0EAE0CB48CC4F0388013336
:2038E0009BB20380BB4200D8E9E4C94B1B881E2B00D8EAE101233370C64B1B78002B00D14C
:20390000FDE19B21C44B49001B88002718009846FDF702FC9B2328705B0098450FD3BF4B89
:203920009946BF4B984601F0F7FE6420FEF750FF4B4642461A602B780137BB42F3DCB94BD4
:2039400002931B78002B00D0BBE4B74A1370B8E4039B1B78002B6FD14A4601211380B34AA7
:203960001170B34A13600022B24B1A70B24B1D78002D5DD05346197800295FD1AF4BB04A4A
:203980001B7812885B00133A9B184A46138001F01FF9012323705346012219784FE0039BA2
:2039A0001878002800D1C3E6A64B1B882F2B1DD84B461D88BCE601F001FB9B4B1B78002B89
:2039C00000D09CE0337822789A46002A2DD05346002B00D100E7039B1B78002B00D1FBE6C5
:2039E000984B1B882F2B00D8F6E6974C974B1B78002B00D09BE0964B1B889B46904B9A4645
:203A00004B4658461D88534668431988FDF70EFC904B013080B21880EFE68F4B03938F4BFA
:203A200098468F4B04938F4B99464B461D881DE601F010F94B461D805346197822783C20FD
:203A4000B424894B64001B78013B4343874800881B1898B21BB2A34223DA854C2380030007
:203A6000B42477331BB26400A34215DA814C23800300B424EF331BB26400A34208DA7E4894
:203A80000380012901D15B46197033789A469CE7794B79381880F4E70300764CF13B2380F3
:203AA000E6E76938724BFF3880B21880D7E7564A1380FFF704FC431B934200DC2FE64B463E
:203AC000401A85B21D802AE60A210A220A2013E653461A78694C93009B185A4A1B011288AE
:203AE0002E33934200DB66E4644B1A7833789A466BE7534A2F2112880092614A01E5237808
:203B0000002B00D0CEE04B461D8833789A46ADE55C4B1B78002B00D194E5039B1B78002B9E
:203B200000D18FE54EE50122574B1A70FAE54146434B08881A889A46009253086021C82260
:203B4000FEF724FE83B29B465A46414B1A8057E701F080F8002180223A4B317019804B4BB3
:203B60004B4819702A4B520019804A4B59639963D963494B59639963D963484B996259626F
:203B8000FEF7BEFBFEF73CFE01F064F880222D4B34701C803D4B00211C701D4B52001C8016
:203BA0003C4B3B485C639C63DC633B4B5C639C63DC633A4B9C625C62FEF7A2FBE2E701F0EE
:203BC00049F81A4B039A1B781278134300D18BE0224B98460123039A1370314B204A1B88DB
:203BE0000492138053461A78164B18887EE401F0D7FD2B78FFF7E7FB01F00EFEFFF7E7FBF9
:203C0000C6020020E2020020E80200201027000018040020CC020020F202002000300040C9
:203C2000AAAA0000F6030020D4020020EA03002014040020F0020020F90200200501002089
:203C4000CE000020D0030020EC020020D000002098010020E0020020F4030020D8000020BB
:203C6000E4030020160300208E0100200C010020EC030020EE030020F0030020F3030020DF
:203C8000FF070000FA0300200E010020D2030020442B0020002C0140000400400044014018
:203CA00020010020FA201E4B80001988FEF780FDFA234A469B00C3189BB21380FA22D200BC
:203CC00093420BD000F084FF7CE6164B117001800293FFF7F6FA00F0BDFF6EE601F06EF929
:203CE000337822789A4670E6FFF7A2F90E4B984642460E4B13800E4B0E4A5A626AE701F05E
:203D00000BFD1CE600240598211CFDF797FB0A4B002801D01C6095E4059A1A6092E4C0463D
:203D2000E8030020F6030020D8000020102700000040014088130000FC030020274B1A78F1
:203D4000002A1DD1B420264940000B8801331BB283422BDA0B80B421224A49001388013386
:203D60001BB28B4200DB0023B42113801E4A4900138801331BB28B422EDB0023138014E076
:203D8000174A1388013B19B21B0411D41180154A1388013B19B21B0413D41180124A1388FC
:203DA000013B19B21B0415D4118070470A80D2E76823FF3313800B4A1388013B19B21B0403
:203DC000EBD56823FF331380074A1388013B19B21B04E9D56823FF331380E6E710010020B5
:203DE000EC030020EE030020F003002070B5164E164B756A1D8000237362154B2D041A88FF
:203E00002D0C500080184019801084B21C80114B64081978FDF70AFA0F4A83B2E41A138056
:203E20000E4BA4B21C80201A736A5B1B9842FBD8FFF7FEF800220A4B1A800A4B1A700A4ACD
:203E400013680133136070BD004001400A040020D8000020D2000020E40200201004002040
:203E6000F6020020F002002014040020F0B5DE464E4645465746E0B58DB002F0B5F802F0F8
:203E8000EFFB012310268020E34A4000116A19431162116A31431162116A01431162DF49CB
:203EA0000D6A1D430D620C6A34430C620C6A204308628020146A40012043106264201064F2
:203EC0000868184308601168194311608021506C090201435164516919435161D04A116AAB
:203EE00019431162116819431160CE4A116819431160516919435161D1681943D160D16888
:203F00009943D160C84A116819431160516919435161C64A11681943116051691943516156
:203F2000C34A116819431160516919435161D1680B43D36001F072FD01F01AFD01F03EFD18
:203F400000230B93BB4BBC491868FDF7E5F80301181A0A218000FDF7DFF80B900B9B002B2C
:203F600005D00B9B013B0B930B9B002BF9D1FEF78FFCB249B2480B78C2789A4201D100F081
:203F800007FEC3704B780C2203710231053003F015F9FEF759FEAB4BFA211B78AA4D013BF8
:203FA0005A1E9341A94A28881370A94BC9001C88A84B60431C80FDF739F9FA21A64BC90001
:203FC0001B781B182B80A54B18886043FDF72EF9A24B1880A24B1C80A24B1B78002B01D197
:203FE000A14A1370A14B1B78002B01D000F0A3FD9F4B03939F4B04939F4B05939F4B089340
:204000009F4B099301F0F4FA00229E4B1A8002F0A5F89D4B9D4A1A60FEF700FC01F0A2FE3C
:204020009B4B1B78002B02D001239A4A13709A4A9A4913689A4D1B051B0D13600B601268B6
:20404000984B120C80211A60002349018A425B41E5225B429343944AE6331370934B944CBD
:204060009846944B944F9A46874B884A1A600023924A1370039B924A1B78012B00D1BDE178
:204080001278002A00D05CE28E4B188843461880FA222B689200934200D957E1002800D1A4
:2040A0003AE1642B00D953E16F4B1E78002E00D14AE19F2800D836E1834B1B789C46002BAB
:2040C00000D137E1C8235B00984200D21CE27F4B1B7899466246642353434A4601335A43A5
:2040E0002178914204DD059B1B78002B00D09CE2002E00D132E11D2800D95BE200233B807C
:20410000734B1B789900C9188900884200DB5DE2704B1B78002B38D03B88302B00D840E1CF
:204120006D4A1278002A00D13BE1313B572B00D9D6E36A4B1B78002B01D000F03DFCFFF744
:20414000FDFD674B67481B7819009946FDF76EF83B880600494664489B46FDF767F878224D
:204160003021330000905846FEF710FB5F4B18800004000CFEF722FB96205C4B80001988AB
:20418000FDF754F85A4B18806EE7534659481968FDF74CF8584B0A211B7858434300C01843
:2041A0004000534B80B21880FCF7B6FF534B80B21880049B1B78002B00D028E2504B1878E5
:2041C000504B1978884200D914E22B68632B00D99DE14D4B1B880C220C204C490A70632B70
:2041E00003D802230220494A1370FA23484A5B0012889A4202D2454B40001870454B1B78B8
:20420000002B00D130E13C4B1B78002B00D019E1064B5B6A28E7C046002C014000040040A6
:204220000044014000200040004801400040014000100040B8010020400D0300C01000083E
:2042400020030020100300208C01002010010020CE00002098010020040100209601002087
:2042600094010020DA0000200D040020D4020020F80200201801002092010020220100201F
:20428000880100201804002000300040AAAA0000120300200E04002000580140D002002083
:2042A00014040020D802002006040020E2020020F402002018030020D00300200104002035
:2042C00013030020E80300200C030020D60000203401002000040020E602002011030020C3
:2042E00026010020581B00002A030000900100201C030020A0860100F4030020D8030020AE
:204300000D030020CC000020D80000200F01002024010020EA0300202070642B1BD8D24BD8
:204320001E78002E10D000232370D04B1B78002B00D0E9E00A23952800D800E1CC4A994619
:20434000137000239C46C5E60026B5E600232370C72800D9A8E600232370A5E6C54B1B7879
:20436000002B00D139E1C44B1B78002B00D025E2C24BC3491E68301CFDF76AF8002800D149
:204380006DE1C04B3B80C049301CFDF74DF8002800D1BDE630233B80BC4B1B78002B00D13B
:2043A000F3E60126BA4B1E70BA4B1B78002B00D115E1B94B1988B94B18780B004000133B0E
:2043C000C018B74B80B218804B1C9946B54B1B885843FCF72BFF4B46181AB34B188000F04F
:2043E000F7FBB14BB14A1B8853639363D363B04A53639363D363AF4B1E7035E61078002820
:2044000000D0A1E0AC4A1278002A00D190E1AB4A12889446AA4A1678FA2276009200B11887
:204420008C4500DCFFE1A74A1678A74A1278B24200D1E9E29F4B1B78002B00D1E3E143469F
:20444000188825E6FEF73EFCA04B1B78002B0BD19F4B1B78002B00D199E19E4B1A889E4B96
:204460001B889A4200D999E19C4B5A6A9C4B9A4200D8F9E59B4B1B78012B00D0F4E522785E
:2044800001322270984A13703B882F2B02D80023944A13700023914A2B609146566A934A7A
:2044A00016804A465362924B36041B88360C5800C0188019801083B29B465A468C4B1A80A5
:2044C0008C4B1978FCF7B2FE8B4B82B21A805B465B089B1A894A9BB21380181A4B465B6A39
:2044E0009B1B8342FAD3FEF7A3FD0023794A1380834A13702B6801332B60B5E55B4B1E78EE
:20450000002E1BD00026002000232370F0E5FA22774B52001B88934200D95CE6794B6421A5
:204520001B6806930A2306980093073BFEF72EF9754BC0B218706E4B1B8850E600206423B0
:20454000FCE6002B00D19FE55C4B1A888323DB009A4271D21300FA21303B9BB289008B42D4
:2045600010D258490E78584908780121891B884200D1FFE165495B0009789BB25B1A4146FD
:204580002F330B802F2A00D959E70023424613805F4A137000232370334B1E78002EADD0DD
:2045A00000232370314B1B78002BC7D00023002023709DE51E2800D1A2E5564B1B789A00B0
:2045C000D21892001100904200DAEDE02D4AA0230092FEF7DBF838809AE5388098E5334A58
:2045E00053639363D363324A53639363D36300F031FB39E50A000126474B0A321B880A395C
:204600005B080096FEF7C2F8444B1880DDE5424E434B444A444936881B88128809880096AE
:20462000FEF7B4F83D4B1880C8E500F013FB00233B8066332370AFE6224B23491B78097882
:20464000994200D189E1394B9C46624453002F4A9BB212789B1A42462F331380EFE6301C42
:20466000FCF70AFF38808EE60D0400200C030020D60000200E04002012030020D40300205E
:2046800000E0FF44FF070000000040420004002011030020F9020020CE00002005010020E8
:2046A0001603002098010020E0020020002C014000040040F3030020D4020020E80300203E
:2046C0002C0100201003002010010020120400202B010020F60200201E01002000400140CF
:2046E000C8AF0000F4030020EA0300200A040020D8000020D2000020E402002010040020CD
:20470000F0020020EC0200200F0100202A010020FA020020340100209401002008010020AF
:20472000960100201201002016010020E8FBFFFFD94B1E88D94B1A78FA2352009B00D11804
:204740008E4200DCA6E0D64BD64A1B7812789A4200D16DE1FA22D44B30000093D2002F23AC
:20476000FEF714F84346FA221880CB4B92001E88CA4B1B785B00D21AB24200DD90E0FA2261
:20478000920094466344B34200DA58E6FDE6C74B1A88C74B1B889A4200D865E60123C54A7B
:2047A0001370FFF723FB5FE6A0231E210093713BFDF7ECFF434638801888A1E4BE4B2F213E
:2047C0001B680693B84B9946BC4B4A461B6807930093069BFDF7DAFF0100B948FCF726FD0E
:2047E000B84B19784908FCF721FDB74B188043461B882E2B00D9D3E0B44BB54A1E60002379
:204800003E801360C8E5FA22A74B60460093D2002F23FDF7BBFF434618809F4B1B889C4611
:204820009E4B1E787600FA229200921B624524DD9C499B4B0E7801211B78C81A864200D1FF
:20484000EBE0A44B1B78002B00D0F8E52F23604600930021944BFDF799FF434680B21880C9
:204860008D4B1B889C468D4B1E78FA2376009B009B1B9C4501DAFFF70BFCFA239B00994639
:204880004E44B44500DDDAE5002342461380914A13707FE6FA239B009A1A964200DB74E677
:2048A0007F4B19787F4B187801235B1A984200D1D5E02F233000009300217B4BFDF766FFF5
:2048C0004346FA2280B21880734B92001E88734B1B785B00D21A964201DAFFF7D9FB4EE729
:2048E00001237D4A1370FFF729FA3B88C82B00D982E07A4B1888FDF761FF794B00229B5EA8
:20490000002B01D0FFF7B0FB764A7749137001220A7076490A70764A76490A8076490A60EF
:2049200076490A6076494A620A222A60694A1370744B754A1B781370744B1B78002B03D013
:20494000099B089A1B881380FEF772FB0121704A53690B435361FFF787FB664908886D4972
:20496000098888423CD85F490978002938D14A4B19800AE65F49088866490988884203D832
:20498000584909780029F2D0002101208C46296056490870604643490E705F490870E9E5B8
:2049A0004B4B5E491E68301CFCF752FD002800D155E64B463B80E6E401210026584AD36837
:2049C0008B43D360524B5E639E63DE63554B5E639E63DE6300F03AFB3F4B1E70FFF7AFFBB6
:2049E0000121CB1A2F4941480B7001210023017049492B600B7026E60023394A5020138031
:204A0000364A5033138076E7464630803648007800283BD02F4A137011E533480078002831
:204A200000D181E02B4B424619700023138006E5304A1088374A1288904204D8294A127844
:204A4000002A00D19FE00122D31A164A27481370012200230270304A2B6013707AE6254B6A
:204A600018882C4B1B88984204D81E4B1B78002B00D183E0002301209C462B601B4B1870CC
:204A8000084B19706146244B197012E701239A1A044B1A70CEE4C046E80300202C010020E1
:204AA0001003002010010020FF070000F60200201C01002012040020C8000020C400002035
:204AC00000879303260100200204002038010020D4030020F3030020110300209001002001
:204AE000EC03002000040020F4030020EA03002028230000D8000020EC020020DC0300200F
:204B000000400140D70000208E010020FA030020002C014028010020FA02002000E0FF445C
:204B200000200040000400401D490B7041461D4B08801B7887E6FA231B4A9B0013800122A6
:204B40001A4B1B491A70039300230B7019490A70194A04911370194A13700592184A1388FD
:204B6000089232331380174A1388099232331380154A138832331380FFF744FAFA26134B70
:204B8000B6001E8095E6FA26104BB6001E80E1E54C780279944201D0FFF7F3F9FFF7FBF9FF
:204BA00010010020F303002096010020F80200200D04002018010020D000002092010020D0
:204BC000220100208801002020010020E80300209023DB051A6819491140802252030A4391
:204BE0001A608022D2009A621A68154911408022D2020A431A60802292009A621A68114951
:204C00001140802252020A431A60802252009A621A680D491140802292010A431A601A68EF
:204C20000A491140802212020A4303211A60084A13688B4301390B4313607047FFFFCFFF16
:204C4000FFFFF3FFFFFFFCFFFFCFFFFFFF3FFFFF000400489023DB051A681C490320114029
:204C6000802252010A431A6040229A621A6818491140802252030A431A608022D2009A62B8
:204C80001A68144911408022D2010A431A6080229A621A68104911408022D2020A431A60A1
:204CA00080220E4992009A620A688243023802430A6088621A680A491140802252020A43FA
:204CC0001A60802252009A627047C046FFCFFFFFFFFFCFFFFF3FFFFFFFFFF3FF000400489D
:204CE000FFFFFCFF00B5062841D8AC4B80001B589F46AB4B1B78002B00D03DE19023DB05BB
:204D00001A68A8491140802252010A431A6040229A629023DB051A68A3491140802292032C
:204D20000A431A601A68A14911408022D2010A431A6080229A621A689D4911408022D202E6
:204D40000A431A60802292009A62032099490A688243023802430A6088611A68964911409C
:204D6000802252020A431A60802252009A6200BD8B4B1B78002B00D0ECE09023DB051A6884
:204D800088491140802252010A431A6040229A629023DB051A6884491140802292030A4320
:204DA0001A601A68814911408022D2010A431A6080229A611A687E4911408022D2020A43A6
:204DC0001A60802292009A6203207A490A688243023802430A608862BFE79023DB051A687E
:204DE00070491140802252010A431A6040229A621A686D491140802252030A431A608022A6
:204E0000D2009A621A68694911408022D2010A431A6080229A611A68654911408022D2026F
:204E20000A431A60802292009A625D4B614A1B78002B00D087E0032113688B4302390B433D
:204E4000136091629021C9050B685B4A1A4080239B0213430B608AE79023DB051A685149DA
:204E60001140802252010A431A6040229A611A684D491140802252030A431A608022D2002D
:204E80009A62474A1278002A6ED11A68474911408022D2010A431A6080229A629023DB05C2
:204EA0001A6843491140802212030A431A608BE79023DB051A683B491140802252010A4377
:204EC0001A6040229A611A6837491140802252030A431A608022D2009A621A68334911402B
:204EE0008022D2010A431A6080229A6293E79023DB051A682B491140802252010A431A60C8
:204F000040229A621A6828491140802252030A431A608022D2009A62214A1278002A35D19C
:204F20001A68224911408022D2010A431A6080229A629023DB051A681D49114080221203D6
:204F40000A431A6001E7032113688B4301390B43136077E79021C9050B68124A1A40802391
:204F60009B0113430B6013E71A6810491140802212020A431A6091E79021C9050B68094A74
:204F80001A4080239B0113430B60C2E61A6807491140802212020A431A60CAE71073000833
:204FA000DA000020FFCFFFFFFFFFCFFFFF3FFFFFFFFFF3FF00040048FFFFFCFF9023DB055B
:204FC0001A681C4903201140802252010A431A6040229A611A6818491140802252030A43E5
:204FE0001A608022D2009A621A68144911408022D2010A431A6080229A611A681049114092
:205000008022D2020A431A6080220E4992009A620A688243023802430A6088611A680A49EE
:205020001140802252020A431A60802252009A627047C046FFCFFFFFFFFFCFFFFF3FFFFFE1
:20504000FFFFF3FF00040048FFFFFCFF2D4A1378002B3DD19023DB0519682B480840802170
:20506000490101431960402199629023DB0519682648084080218903014319601178002967
:2050800037D11968224808408021C90101431960802199629020C00503681E4919408023CE
:2050A0001B030B43036013781B4A002B1AD1032113688B4302390B43136091629021C90540
:2050C0000B68164A1A4080239B0213430B6070479020C00503680C49194080239B010B43D0
:2050E0000360C2E7032113688B4301390B431360E4E71968064808408021090201431960F1
:20510000C8E7C046DA000020FFCFFFFFFFFFCFFFFF3FFFFFFFFFF3FF00040048FFFFFCFFD7
:20512000F0B5CE4647466E4C80B56368226883B0981A6C4B0100C2186B4B9A423FD86B4D0D
:205140002B78002B50D06A4E3378002B1DD1694B98461B78002B00D1A4E0674A9146108820
:205160004246664F013339881370FDF721FB322800DC76E000232B703B884A46138033788F
:20518000002B0AD061682368C91A5D4B5D4C99425BD923784B2B00D989E000225A4B5B49B5
:2051A0001A805B4B5B4A186812680B88C41A944211DC1C1AA24215DA9B1A0B800DE0002284
:2051C000554B1A80524B18685049524A0B881268C41A9442EDDD9B180B8003B0C0BCB9464C
:2051E000B046F0BD0880F8E74C4B1C78002C11D04B4B1A8890421BD84A4B1988FA239B0082
:2052000000930023FDF7C2FA414B186000223E4B1A80D9E7394B1A88424B1988424B0093AB
:205220002F23FDF7B3FA3A4B2F2856D01860EDE7324B511C1C88FA23DB00009322003B4B6C
:20524000FDF7A4FA324B1860E0E73648237806880133F200921B5118DBB2C90823700180AB
:2052600098E73988226863689B1ACA00521A9B184246DB0812789BB23B80322A00D87CE767
:205280002B4A193B94469BB23B806344DA0FD318212228495B108B540123337000F080FAB9
:2052A0003B886AE7144A80B29146108058E71D4A002613881F4919339BB213801E4A2E70E2
:2052C00094466344DA0FD31820225B108B54FDF7BBFC267000F0A0FA5FE700201C6095E7C4
:2052E000442B0020DFFCFFFF760500001A0400201D0400201C0400201E0400202E0100207B
:20530000E104000022040020F8030020E8030020240400209C01002018040020F8020020E1
:205320003201002030010020FF070000E90300002AF9FFFF2003002012FDFFFFF8B5434C2A
:205340002378002B03D0424B1B78002B06D1414B1B78002B48D0012B07D0F8BD3E4B1B785C
:20536000002B2FD000F0FEFCF7E7394B1B78002B2FD13A4B1B78012B56D0394B1B78012B4C
:2053800043D02378002BE8D1364C2088002833D0354A00251380354B9842DED9344E3188A3
:2053A000FDF706FA322847DC324F3B780133DBB23B70322B03D9304B1B78002B3FD02388B0
:2053C0003380CAE700F016FDFCF7A2FFFDF72CF8C3E7214B1B78002B0BD0FCF799FFFDF78C
:2053E00023F800F0BFFCB8E700F03CFD00F0BAFCB3E700F0FFFCB0E7204B1B78002B18D14B
:20540000194A138801331380A7E7FFF789FE0A211B4A136A8B43136200F0A4FC0421194A54
:2054200013680B431360ACE7FCF7FEFF00F09AFCA3E70D4B188090E70E4B1D70BFE700F0BA
:2054400027FA01220D4B3D701A70B8E7E602002014030020D2030020442C002013030020E0
:20546000F6030020E202002018040020DC050000200400201B0400201D0400201A040020F0
:205480000044014030000240031C0B2800D90B23014A5B001370704728040020F8B5DE46BF
:2054A000574645464E460320E0B5FFF71BFC434B00249A46424B434D9B4616E069780029DB
:2054C00038D1414BE001001B596340009963D9633E4B8019596380B29963D963FDF778F95A
:2054E00000243B4B02359D420ED05B46394A1A60002352462E781380FF2EDFD1344B0134EB
:205500000235E4B29D42F0D1FFF7A4FB002332492D4809882D4A83629362C162D1625246A6
:205520001380274B2B4A1A60F0BCBB46B246A946A046F8BD4B015B1ADB00591AFA231B0100
:205540009C4626486144FBF771FE1F4B010099460A234A4693621D4A070093622048904658
:20556000FBF764FE4B46D8624346D8621D4B1E491B785843FBF75AFE4B4658639863D86380
:20558000434658639863D863E001001B40008019FCF7E4FD041CB8B2FCF72EFE011C1348C7
:2055A000FCF720F9011C201CFCF7E4FAFBF764FF80B2FDF70DF9002493E7C046F803002075
:2055C0000030004054030020002C014000040040D0030020AAAA0000CE0000208096980050
:2055E000003E490028040020CF07000000007A4470B572B61E4B1B78FF2B09D0FFF74EFFB5
:205600001C4B1D4A1B88D3621C4AD36262B670BD194D1A4C1A4B0320EB62E362194B1B7827
:205620006B63AB63EB636363A363E363FFF75AFB3723C820AB62A362FDF7CAF80520FFF7BE
:2056400051FB2823C820AB62A362FDF7C1F80620FFF748FB1923C820AB62A362FDF7B8F8D3
:20566000FFF7F8FA0023084AAB62A3621380C7E7307C0008CE000020002C01400004004027
:20568000CF07000028040020F8030020F8B51A4B1A4D1B4CEB62E36272B63C23194E1A4F04
:2056A00001203760AB62A362184B1B786B63AB63EB636363A363E363FFF714FB4B20FDF78A
:2056C00087F850234B20AB62A362FDF781F85A234B20AB62A3623760FDF77AF8FFF7BAFA4D
:2056E00000230B4AAB62A36213800A4B1B88EB62E36262B6F8BDC046CF070000002C0140ED
:205700000004004000300040AAAA000028040020F8030020CE00002070B572B6184D194C15
:20572000194B1A4AEB62E362194B03201A605023AB62A362174B1B786B63AB63EB636363A4
:20574000A363E363FFF7CEFA6420FDF741F846236420AB62A362FDF73BF828236420AB628C
:20576000A362FDF735F8FFF775FA00230A4AAB62A3621380094B1B88EB62E36262B670BDB4
:20578000002C014000040040CF070000AAAA00000030004028040020F8030020CE00002069
:2057A00070B5154B154D164CEB62E3623223AB62A362144B02201B786B63AB63EB636363A3
:2057C000A363E363FFF78EFA9620FDF701F80E4A0E4B96201A601E23AB62A362FCF7F8FF3E
:2057E000FFF738FA00230A4AAB62A3621380094B1B88EB62E36270BDCF070000002C01406C
:205800000004004028040020AAAA000000300040F8030020CE00002070B5154B154D164CE2
:20582000EB62E3622823AB62A362144B02201B786B63AB63EB636363A363E363FFF752FAE7
:205840009620FCF7C5FF0E4A0E4B96201A605023AB62A362FCF7BCFFFFF7FCF900230A4A65
:20586000AB62A3621380094B1B88EB62E36270BDCF070000002C01400004004028040020FA
:20588000AAAA000000300040F8030020CE000020F0B5C646194B1A4E1A4D00B5F362EB6200
:2058A00072B6194B77241B78184F7363B363F3636B63AB63EB63164B9846434614211F60DF
:2058C0002000FBF7B3FCFFF70DFA63100A33B3620A20AB62023CFCF77BFF631CEDD1FFF730
:2058E000B9F900230B4AB362AB6213800A4B1B88F362EB6262B680BCB846F0BDCF0700005A
:20590000002C01400004004028040020AAAA000000300040F8030020CE0000200D4885469D
:205920000D480E490E4A002302E0D458C4500433C4188C42F9D30B4A0B4C002301E013604E
:205940000432A242FBD301F0E7F8FCF7B5FCFEF78DFAFEE700400020C0000020BC0100206D
:205960004C730008BC010020582C0020FEE70000C2210C4B89005A580B4802405A508022A4
:2059800092001A60094B0A4A0A499A600A4ADA605A68120C12040A4301215A601A680A438A
:2059A0001A60704700E100E0FF00FFFF0800024040240140881300002C0400200023154A9C
:2059C00082B0019393681449194080231B060B4393609368002BFCDB01230193019B002BCF
:2059E00005D0019B013B0193019B002BF9D1094A094993680B4001210B43936013681942B1
:205A0000FCD0936804490B4004210B43936002B07047C04600240140E8FFFF7FF0B5CE46CF
:205A2000474680B593B01022002102A8FCF768FC1422002106A8FCF763FC102200210EA8AD
:205A4000FCF75EFC80204A4B8000996990240143996180219A69890202400192019A5A69EE
:205A6000E4050A435A615B6901220B400093009B03230CA9200000250C920D9301F080F80E
:205A8000022203230CA920000C920D93109501F077F8042203230CA920000C920D931095A0
:205AA00001F06EF8082203230CA920000C920D93109501F065F82F4B2F491A682F4C0A4000
:205AC0001A601A682E4900260A4020211A601A6800270A431A601A6820318A431A601A681C
:205AE00040310A431A601A68264920001140802252000A431A601A68234911408022D2009E
:205B00000A431A600122A36A91461343A362A36A0732904613438022A3621023120602A94D
:205B2000029203930496059700F0F8FF802201239201089209930722069607970A95E36842
:205B40000435AB43E3606369200093434A461343636106A900F0FCFF42466368AB436360D1
:205B600063689343636013B0C0BCB946B046F0BD0010024008000240EFBFFFFF0024014033
:205B8000FFCFFFFFFFFCFFFFFFF3FFFF7047C046F0B54746CE4680B585B016006A46CB0F43
:205BA0005B185B1098465B000733DB08DB00D31A00AF9D466D460C00814642460021280000
:205BC000FCF79EFB012C0BDD484600234178027809025C000A4301332A5302309845F5DCFB
:205BE000434601212C4A7B60D3681942FCD113691B0605D5294B1B685360294B1B6853607B
:205C0000B30517D10221244A13690B431361566113693E310B4313613F39D3681942FCD1D6
:205C20002023D1680B4200D0D36002211A4A13698B4313610023BB60FB60FB687A689A4299
:205C40001FD90120202414490B6903430B61FA68BB685200525B9B191A80CB681842FCD138
:205C6000CB681C4200D0CC600B6983430B61BB680233BB60FB680133FB60FA687B689A426B
:205C8000E2D38021BD46044A13690B43136105B0C0BCB946B046F0BD00200240A001002029
:205CA000A401002070B5002A2BDD040003230C4323405C42634102244D1C451BAC42A441E8
:205CC00064421C421ED0531E082B1BD90B009408A4006418451A1E68EE500433A342FAD169
:205CE00003241300A34314420BD0CC5CC4545C1CA24206DD0D5D023305559A4201DDCA5CFB
:205D0000C25470BD8A18451A0B786B5401319142FAD1F6E780220D4B9202D9680A43DA60FA
:205D2000DA680B490A40DA6001210A22094B99611A62094A12789A62084ADA625A690A43BA
:205D40005A610022064B1A707047C04600100240FFFFFDFF00440140B4010020FFFF00002A
:205D6000442C00208022184B9202D96817480A43DA60DA6816490A40DA600A210122154B00
:205D80009A6119621449097899621449D96259691143596100210170596211481149C86024
:205DA00011488860114800684860114808608021D86889000143D960196A114319621968BE
:205DC0000A431A607047C04600100240442C0020FFFFFDFF00440140B4010020FFFF00000B
:205DE000442B00203000024034440140AC0100208B090000134B14491A78144B14489A6284
:205E00003D22DA623C3A0A705969114359611149C86011488860114800781730486010484C
:205E200008608021D86889000143D960196A114319628021586C09020143596419680A4382
:205E40001A607047452C0020442C0020004401402C0200203000024034440140402B002067
:205E60009B090000F0B54F464646D6464B4B4C4CC0B59A461C604B4B4B4D9C4600236246C2
:205E800013604A4A290013709146494A0026904600200027137008C97C350A689A4206D079
:205EA000D31A9C4201D91C0001270126C018043113008D42F1D1002F45D05346A21E1C6008
:205EC0002300002E47D0614640090860012A0DD8312844D9374B9C466444631E9C41364B91
:205EE0001C70E0BCBA46B146A846F0BD221F032A17D83128EED8012249460A702F490A704E
:205F00002F490A702F4A304951622C212F4A11702F4A3049116007212F4A11702F4A19315B
:205F200011602E3B2E4AFF3B9342D3D80123424613702F22214B1A702A4B0C3A1A80274B18
:205F4000213A1A60C6E7002E22D06346144C400918602300E5E761460E60012A14D8002298
:205F600016490A7016490A70494601320A702C21164A1170184A23391170154A1549116098
:205F80002021164A1160CCE7221F032AB3D9C8E76346034C1E602300C3E7C046482C0020B6
:205FA000204E00003C2B0020442B002013030020F6030020E0B1FFFFD2030020B4010020B5
:205FC000452C002000440140FFFF0000A8010020B0010020E8FD0000402B0020AC010020D6
:205FE000F24C0000D400002000B51B4B1B4883B01B4A9A1802CB11608342F9D10123032093
:20600000184A916919439161926913400193019B154B196881431960FA211A6889000243CF
:206020001A60124B1868FBF777F8802301385B04984200D3FEE7C0210D4A090650600D488F
:20604000036A1B021B0A0B430362002393600733136062B603B000BD00100008C0100008A3
:2060600000F0FF170010024000000140B801002010E000E000ED00E00121334A10B5136832
:206080008B430B4313601368304A13680B431360013113681942FCD0F82113688B43783959
:2060A0000B431360536B7F390B435363274A0131536B1942FCD0F821536B8B4378390B4379
:2060C0005363536A7F390B435362204A0131536A1942FCD053681E491940A0239B030B43E8
:2060E0000F215360D36A8B43D362802311685B040B4380211360154A890413680B42FCD020
:20610000F0215368114C8B435360536811490B400321536053688B4301390B4353600C22AC
:2061200063681340082BFBD10B4801F031F80A4801F03EF80422636B93436363236B013A03
:206140009343236310BDC0460020024000100240FFFFC2FFFFF8FFFF006CDC02094B0A4AB6
:2061600007211A60094A1A6002225A60FA2212019A60DA681142FCD1054A1A61054A1A60B4
:206180007047C04600300040CCCC000055550000FF0F0000AAAA0000F0B5DE4657464E4634
:2061A0004546E0B59DB01422002103A8FCF7A8F82022002114A8FCF7A3F81822002108A825
:2061C000FCF79EF8182200210EA8FCF799F880225B4F1201BB695B4E1343BB61BB6903A933
:2061E00013400293029B584B30009046059300F0F7FD80223368002413433360B368534AF3
:2062000000251340B3606022002308211492159316941795189419951A941B954C4B8B4661
:206220009946B36930000B43B36114AB1A00073900F020FE0421B3698A468B434146B36130
:20624000B36930000B43B36114AB1A00102100F011FEB3693F4A59461340B3614B465B6888
:2062600030000B4349464B60802114AB1A00490000F000FE4B4651465B6870228B434946DB
:206280004B6073682C2193437360B368103213436A46B3600023521813706A46D385802252
:2062A0000A930023920108A930000C920D930894099500F0E7FE80217A6989020A437A6126
:2062C0007B6900260B4080210193019B7A69C9020A437A617B6980220B400093009B02239E
:2062E000D2000E920F9390230227DB050EA918009846109411951296139700F041FC8022B6
:20630000022392000EA940460E920F93109411951296139700F034FC8022022352004046EC
:206320000EA90E920F93109411951296139700F027FC1DB0F0BCBB46B246A946A046F0BDC1
:2063400000100240002C0140CF070000F8BFFFFF182C0140FFFBFFFFF0B5C646022500B5E9
:2063600094B01422002101A8FBF7CAFF202200210CA8FBF7C5FF1822002106A8FBF7C0FF97
:20638000464B474CDA6901A92A43DA61DB6920002B400093009B434B8027039300F020FD6F
:2063A00080222368042613432360A3683E4A7F001340A360602200230C920D93002310959A
:2063C00012970F93A369583A13439046A3610CAA0121200000F04EFDA3691021B343A3613A
:2063E0008023A2691B011343A3610CAA200000F041FDA3692D4A2E4D13404246A3616B68C5
:20640000390013436B600CAA200000F033FD702207216B680127B3436B60A36800259343B0
:20642000A360A3688B433343A360E36839318B43E360E3681F4900260B40E360636806A960
:2064400093436360402202230692079390230024DB0598461800089409950A960B9700F0D1
:206460008FFB8022022306A9404606920793089409950A960B9700F083FB0122022306A983
:206480000D4806920793089409950A960B9700F077FB14B080BCB846F0BDC0460010024094
:2064A00000040040CF070000F8BFFFFFFFFBFFFF18040040FFBFFFFF0004004880201C4BAA
:2064C0008002596910B50143596180215A6988B002400192019A5A69C9020A435A615B694F
:2064E0000C220B400093002105A8009BFBF708FF8023104880228362012302920393032338
:2065000002A9049300F03CFB1022012302920393032200239024049205930023E40520003C
:2065200002A9069300F02CFB1023A36208B010BD001002400004004830B58FB0142200212A
:2065400003A8FBF7DDFE0C2200210AA8FBF7D8FE8020394B800299698025014399618021CE
:206560009A69C90202400292029A5A6933480A435A615B6980220B400193019B022352003D
:2065800008920993022308A90D9300F0F9FA2C4B2C491A68C2200A401A601A682A498000E3
:2065A0000A4020211A601A68284C8A431A601A6820318A431A601A682549AA432A431A60BB
:2065C0001A681140802252000A431A601A6821491140802212010A431A601F4B1F491A5830
:2065E00011408022D2030A431A508022D2001A6000236A4693813F2205926A46200003A9D3
:2066000004930693137700F0EBFB03222368AB432360A3699343023A1343A361A3690B3208
:206620009343A361A369E4329343A361236AE63A134323620FB030BD0010024000040048B2
:2066400030000240EFBFFFFFFFCFFFFF00440140FFFCFFFFFFF3FFFF00E100E0FFFF00FF24
:20666000F0B5DE4657464E464546E0B501258DB0FFF702FD80216B4C4905A36917262B434B
:20668000A361A36980272B400293029BE2690A43E261E369644A0B4010210193019B1368AA
:2066A00088460B431360FFF709FFC221636989002B43636163695D4A1D4000955C4D009B3A
:2066C0006B581A408023DB0313436B508023DB002B60FFF761FDFFF73FFE1422002107A875
:2066E000FBF70EFE8021E26949000A43E261E3690B400693069BC4239B0099464A46EB58D2
:2067000007A91B021B0AAB5080231B032B606B469E8300239B460893FA231B0109935B4659
:206720000A93444B9A46180000F05AFB534652461B6800213B43136007A81422FBF7E0FD76
:206740008021A26949020A43A261A3690B400593059B6B469E83384E384B07A930009A46C8
:20676000099300F03DFB3368354ABB433360B368002113407022B360736807A89343736043
:20678000B3685C3ABB43B360FBF7BAFD4246E3692F261343E361E36907A913400493049B46
:2067A0004B46284AEB581A4080231B0213434A46AB5080239B022B606B469E835B46224DEB
:2067C000089328006433099300F00AFB2B681422BB432B60AB680021BB43AB6007A8FBF79E
:2067E0008FFD8021A269C9020A43A261A369174C0B400393039B6B469E83534607A920001D
:20680000099300F0EDFA2368BB432360FFF794FE00F01EF80DB0F0BCBB46B246A946A04634
:20682000F0BDC0460010024000200240FFFF00FF00E100E00020004000400140FFFF000054
:20684000F8BFFFFFFF00FFFF001000400048014030B5002591B01C22002108A8FBF750FD14
:206860008020474B05959969C0010143996180219A69C90202400192019A5A69414C0A43CF
:206880005A615B6940220B400093009B022302920393032301220493002302A93A48069287
:2068A000079300F06DF92368384AC62013401022134323602368364AC02113402022236093
:2068C00023688000934323602368203293432360236840321343236023682E4A09061340E3
:2068E000236023682C4A13402C4A236013581B021B0A0B43135080231B051360E12200230E
:20690000120308920993002200230A920B93082200230E95224D08A928000C920D9300F047
:20692000DBFBAB681F4A20481340AB606B681F4A1F4913402A226B60AB689343AB602B68AA
:20694000293A13432B6023681A4A0340102B13D0A160E2600B4B18495A680978120C120432
:206960000A4302215A601A680A431A601A6806310A431A6011B030BDE160A260EAE7C0465C
:20698000001002401C00024000040048EFBFFFFFFFCFFFFFFFFCFFFFFFF3FFFF00E100E0D9
:2069A00000380140FFFBFFFF10400000FFB7FFFF4C2C002028380140B50100207047C04696
:2069C000FEE7C0467047C0467047C0467047C0468022164BD200196810B5114203D01449F7
:2069E000097800290AD1114B1A68920512D41A68120502D5802252005A6010BD0A240D4849
:206A0000016AA143083C214301625A60074B1A689205ECD58022012152005A60064A13689B
:206A20008B431360FEF78AFCE7E7C04600000240F603002000440140300002407047C046B7
:206A4000014B5B697047C04600040140054B10B51A69D20700D410BD022252421A61FCF7EC
:206A6000F9FBF8E700100040022210B5024B52421A61FCF7B9FB10BD002000407047C0461D
:206A80007047C046074B1A69920702D5032252421A61044B1A69D20702D5022252421A610B
:206AA0007047C04600400140074B1A69920702D5032252421A61044B1A69D20702D5022279
:206AC00052421A617047C04600040040084B10B51A68920706D40822054B19680A4200D082
:206AE0005A6010BD01225A60FFF750F8F3E7C04600000240074B1A69920702D503225242D4
:206B00001A61044B1A69D20702D5022252421A617047C046002C01407047C0468268030071
:206B200010B50120D20710D48C684A68D8682243CC6809682243054C204002430020DA600D
:206B40001A69920092080A431A6110BDC73FFFFF8368020010B50120DB070ED44C680B682F
:206B6000D06823438C682343CC68096923430B430249014000200B43D36010BD3CC2FEFFCE
:206B8000F0B5DE4657464E464546E0B50A684B6883B0002A00D172E09C46012301245B426E
:206BA00063449846A34600230AE00E69C56874434E4635402C43C46014000133DC4041D0EE
:206BC0005C4615009C4025402242F5D02C006C436700BA46A2445746FF43B9465746066883
:206BE000BE43674667433E4306604646012EDCD88668B2468E685746664301964E46374023
:206C00003E00019F37438760C6684F46B2460E6966430196564637403E00019F37436646AC
:206C2000C760022EC8D1FF2D1DD86443056A2601361BB5434E69013374432C430462140032
:206C4000DC40BDD14346012B05D84368C96893434A431A434260002003B0F0BCBB46B24642
:206C6000A946A046F0BD2D0A6D436D43446A2E01761BB4434E697543254345629CE7013B59
:206C80009846DFE70C23184A70B5516805000B40082B11D0154B14492B604A68144812060F
:206CA000120F825CD3406B604A6812495205520F8A5CD340AB6070BD802350685B021840F1
:206CC000434258410C4B40421840084B0F249C46D16A6044214001315668FAF71DFAB30C06
:206CE000234002334343D6E70010024000127A002C7300083C73000800F7C2FF030070B59D
:206D00000020002B33D1314A0333116B0B40022B52D0032B48D05168012B29D00C230B40BF
:206D2000082B51D1802350685B02184043425841274B40421840274B0F249C46D16A60441E
:206D4000214001315568FAF7E7F90300AD0C2C40A01C58431D4B20495A685B681206120F04
:206D60008A5C5B05D0401D4A5B0FD35CD84070BD0B330B40082B1DD1802350685B021840BE
:206D800043425841124B40421840124B0F249C46D16A6044214001315568FAF7BDF9AD0C9D
:206DA0002C4002346043E2E713680222100018401A42DCD00748DAE71800126A104013426D
:206DC000D5D080200002D2E70248C3E70010024000F7C2FF00127A002C7300083C730008CB
:206DE0001D4A0368904226D08022D205904219D01A4A904216D01A4A904217D0194A904257
:206E00001DD0194A90421AD0184A904217D003608B68C3620B88836201224369134343618F
:206E200000207047702293434A681343104A1340CA681343EBE7702293434A6813430C4A3E
:206E40001340CA68134303608B68C3620B8883620B7C0363E0E7C046002C014000040040F9
:206E600000200040004001400044014000480140FFFCFFFF802370B55B00994200D1ADE0CE
:206E800041D8012900D171E010296DD1036A714D8B430362036A466884692C4015682D0298
:206EA0002C432025AB431D0013691B012B438B4351680D0168492B43884208D0674988423D
:206EC00005D06749884202D06649884214D180218B431D00536940399B012B438B439168A1
:206EE0008D0161492B430E409169604D890031432940D569EE000E43D2684660846182636A
:206F00000362002031E080235B0199422CD1016A574E504C31400162036A4568C1692140DF
:206F2000146824020C435349194013691B030B435168334009030B434749884208D047493B
:206F4000884205D04649884202D04649884204D149490D40916989010D43D2684560C46182
:206F600002640362002000E0012070BD7326036A8B430362036A44688569B54316683543CA
:206F80000226B343166933438B4351680B433249884208D03149884205D03149884202D0BD
:206FA0003049884213D108218B43190053699B000B4304218B43916889000B432F490C406E
:206FC00091690C432E490C40D16949000C43D26844608561426303620020C6E77324016A36
:206FE000264E31400162036A4168C569A54314682543234C1C4013691B0223435468334040
:2070000024021C43144B984208D0144B984205D0134B984202D0134B984213D1134B144EE6
:207020001C4053690E409B0223430F4C23409468A4021C43936919010E4B31431940D369B0
:207040005E013143D3684160C561C363046200208BE7C046FF8CFFFF002C014000400140C0
:207060000044014000480140FFFBFFFFFFF7FFFFFFEFFFFFFFDFFFFFFFBFFFFFFFFEFFFF97
:20708000FFFDFFFF8A680B7B13430D4A13404A6813430C4A13400A6813430B4A1A40CB8902
:2070A00013430A4A13400A691343094A13404A69084913430B401343436400207047C046E5
:2070C000FFFBFFFFFFF7FFFFFFEFFFFFFFDFFFFFFFBFFFFFFF7FFFFF30B5036804000D0063
:2070E00085B0DB071DD44B68C96802680B4329690B43A9690B4320490A4013430360436895
:207100001E4A1340AA681343436083681C4A13406A69134383601B4B984205D01A4B9842A5
:2071200018D0012005B030BD0020FFF7E7FD0028F7D029680029F4D08023AA691B029A428E
:207140000DD04B081818F9F7E7FF03041B0C0020E360E7E701A8FFF795FD0398E7E74B08AD
:207160004000C018F9F7D8FF084B03400007400F1843E0600020D5E7F369FFFFFFCFFFFFA7
:20718000FFFCFFFF0038014000440040F0FF0000FA2110B58900F9F7BFFF0022034B01384A
:2071A00058609A6005321A6010BDC04610E000E0014B18607047C046B8010020002310B587
:2071C0009A4200D110BDCC5CC4540133F8E70000F8B5C046F8BC08BC9E467047F8B5C04669
:2071E000F8BC08BC9E467047B819000844190008A018000858180008A018000880190008A5
:20720000A018000858180008441900084419000880190008581800085E1800085E18000857
:207220005E1800088E1900084419000844190008A018000854180008A018000880190008C2
:20724000A018000854180008441900084419000880190008541800085E1800085E1800081F
:207260005E1800088A190008181C0008E81B0008E81B0008E61B0008EC1B0008EC1B00086C
:20728000341D0008E61B0008EC1B0008341D0008EC1B0008E61B0008E01C0008E01C000804
:2072A000E01C0008701D00086A260008102700080A270008042700086A2600086A260008C2
:2072C0006A260008F2260008DE260008D6260008CE2600086A260008C8260008B42600087A
:2072E000A22600086A2600086A2600086A2600086A2600086A260008942600086226000874
:20730000191B12131D1516171A090A0B1E0D0E0F6E4D0008704D0008DA4D0008B04E000878
:20732000584E0008EE4E0008F24C00080000000000000000010203040607080900000000ED
:2073400001020304F9100008D1100008CA00000010270000E8030000FF00CF07010206005F
:20736000E8030A05D4300100000000002003000000000000E8030000000000000000000000
:207380000000000000000000204E0000A08601000D0A0A00CF070200B4000105010046005E
:2073A0004A011400010201000600060090010D00D0070EFFDC05010164006C074C04DC05F1
:2073C00005050000000000000A000000000000006400000000000000000000000000000035
:2073E000000000001027000050C3000000000000020000000000000032000000000000000F
:207400000000000000000000000000001027000050C300000D006419390101006400011EDA
:20742000CF079001CF07D007FA00000023016745AB89EFCD2C0000002000000024F400001A
:207440000A0A000000127A00FFFFFFFFFFFFFFFFFFFFFFFFFFFFFFFFFFFFFFFFFFFFFFFFA4
:20746000FFFFFFFFFFFFFFFFFFFFFFFFFFFFFFFFFFFFFFFFFFFFFFFFFFFFFFFFFFFFFFFF2C
:20748000FFFFFFFFFFFFFFFFFFFFFFFFFFFFFFFFFFFFFFFFFFFFFFFFFFFFFFFFFFFFFFFF0C
:2074A000FFFFFFFFFFFFFFFFFFFFFFFFFFFFFFFFFFFFFFFFFFFFFFFFFFFFFFFFFFFFFFFFEC
:2074C000FFFFFFFFFFFFFFFFFFFFFFFFFFFFFFFFFFFFFFFFFFFFFFFFFFFFFFFFFFFFFFFFCC
:207C0000010201015C417264754265652020202020000000010101021864370E0000050000
:207C2000808080320032004F4553432366303531FFFFFFFFFFFFFFFFFFFFFFFFFFFFFFFF27
:207C4000FFFFFFFFFFFFFFFFFFFFFFFFFFFFFFFFFFFFFFFFFFFFFFFFFFFFFFFFFFFFFFFF44
:207C6000FFFFFFFFFFFFFFFFFFFFFFFFFFFFFFFFFFFFFFFFFFFFFFFFFFFFFFFFFFFFFFFF24
:207C8000FFFFFFFFFFFFFFFFFFFFFFFFFFFFFFFFFFFFFFFFFFFFFFFFFFFFFFFFFFFFFFFF04
:207CA000FFFFFFFFFFFFFFFFFFFFFFFFFFFFFFFFFFFFFFFFFFFFFFFFFFFFFFFFFFFFFFFFE4
:020000040801F1
:00000001FF
